S00E0000626C696E6B792E737265638D
S11300000BC023C022C021C020C01FC01EC01DC001
S11300101CC01BC01AC019C011241FBECFEDCDBF18
S113002010E0A0E6B0E0E8EEF0E003C0C895319639
S11300300D92A036B107D1F710E0A0E6B0E001C000
S11300401D92A036B107E1F735C0DACFCF93DF9325
S1130050CDB7DEB728970FB6F894DEBF0FBECDBF7D
S11300606D837E838F83988719821A821B821C82F8
S11300700BC089819A81AB81BC810196A11DB11D00
S113008089839A83AB83BC8329813A814B815C81C8
S11300908D819E81AF81B885281739074A075B0790
S11300A044F328960FB6F894DEBF0FBECDBFDF91A0
S11300B0CF910895CFEDD0E0DEBFCDBFEAE3F0E00D
S11300C08FEF8083EBE3F0E08FEF808368ED79E5D9
S11300D080E090E0BBDFEBE3F0E0108268ED79E5CF
S10B00E080E090E0B3DFEECFF5
S9030000FC
